:030000000219FDE5
:03000B000200AA46
:03002B0002018748
:03005B0002033964
:030073000203265F
:1000800002030406080C10182030406080040608A3
:100090000C10182030406080A0C00003070F1F0D17
:1000A0000D0403060D0503030202C2AF306308C24C
:1000B0006385798AD2AF32C0D0C0E0206221E525C5
:1000C0006016E473E525F4C3334009758A00D263F2
:1000D000F57901D6F58AD262D0E0D0D0D2AF32C362
:1000E000E526334009758A00D263F57901F0F58A77
:1000F000C262E526F4602F30682520720DD0E0D072
:10010000D0C292C296C294D2AF32C292C296C29468
:10011000206F0C206509740ED5E0FDE57B4290D080
:10012000E0D0D0D2AF32758A00D263757900C28D2B
:10013000D262211F01C4306805206502D29201C439
:10014000306805206502D29401C43068052065023C
:10015000D29601C4C29330680A2065077410D5E0B6
:10016000FDD29201C4C29530680A2065077410D58B
:10017000E0FDD29401C4C29730680A20650774106C
:10018000D5E0FDD29601C4C2AFC2AD53E6EFC0D0F8
:10019000C0E0D2D3D2AFE57A6009E5776005757724
:1001A000004129757701C2CEE52A600720744F15FA
:1001B0002A21FE7800790020742EE580307E01F43B
:1001C00030E50278FF53DACF207E0343DA20307E19
:1001D0000343DA10C2D8C271E580307E01F430E505
:1001E0000279FFC3E89970CB306103752A4020740F
:1001F00003752A40885CD270E86003755F00207444
:100200000DE52B6004152B410E43DA01C2D8207096
:10021000024121A85C206102C270207402411F8843
:10022000227882B6040385222420CF0AD0E0D0D0E1
:1002300043E610D2AD32C2CF053AE57A6009E578DF
:100240006005757800611C7578017802E52A600503
:10025000307402152AC3E55C94014005755F0041C6
:1002600072756000756900E55F2401F55F500375E4
:100270005FFF7982B7020D306E1DC3E522943240D4
:1002800016854C227982B7030E306E0BC3E522949B
:10029000324004798E8722C3E5239522600840040A
:1002A000152341A60523D8CA0569E56970021569B9
:1002B000D56A69756A017808E56B60497805C3E518
:1002C00069956B4057C3E569956C50087801756A6C
:1002D000030202E0C3E569956D50057801756A0176
:1002E000C3E5629524401E7982B704026111206E35
:1002F00014852462E569046003856B69756A01757C
:10030000233C02031CE5622850057562FF6111F56C
:1003100062E5620470067560FF7569FFD0E0D0D0B9
:1003200043E610D2AD32C2AF53E67F7592FA7593B1
:10033000FFC260759104D2AF32C2AF53E6EFC2ADD7
:10034000C0D0C0E0C0F0D2D3D2AFA8FBA9FCE57A00
:100350006007C3E913F9E813F8C2D830710261AB42
:1003600053DACF207E0343DA10307E0343DA20D203
:1003700071E580307E01F420E502618288278928BA
:10038000A19053DACF207E0343DA20307E0343DA94
:1003900010C2D8C271307402A17C7800E580307E32
:1003A00001F430E502A17C885CA16453DACF207EA1
:1003B0000343DA20307E0343DA10C27120610281E8
:1003C0008453DACF207E0343DA10307E0343DA20F1
:1003D000C2D8D27188578958C3E89555F8E995561F
:1003E000F97B007E087A00C3E8948CE994005005FC
:1003F000755B008176882178A2E6A8216055C3E864
:1004000094C8E994005008E4D2E4FB7A0A8151C30D
:10041000E89468E994015008E4D2E3FB7A0F815133
:10042000C3E894D0E994025008E4D2E2FB7A1E813A
:1004300051C3E894A0E994055008E4D2E1FB7A3C6A
:100440008151C3E89498E994085008E4D2E0FB7A1B
:10045000787E00C3E89559FCE9955AFD30E70AEC2F
:10046000F42401FCEDF43400FD755B00C3EC9AED5F
:0D0470009E5003755B018859895A855755C8
:10047D008558567802A164C3E89527F8E99528F9BF
:10048D00307C02A148307B02A148307A02A1412084
:10049D00750281A7E9FDE8FC81C6E9C313F9E813EC
:1004AD00F8307902A141E9C313F9E813F830780265
:1004BD00A141E9C313FDE813FC20612CC3EC941C8E
:1004CD00ED9402400281DDED701EC3EC94C850180E
:1004DD000529E52970021529C3E529940A5002A1C1
:1004ED007C755C00D270A17CE52960021529740031
:1004FD00207F037896E624FAFEE43400FFC3EC9ED9
:10050D00FCED9FFD500678007900A148C3EC94FFE7
:10051D00ED9400400678FF7900A148EC8572F0A4B7
:10052D00C5F0A2F733F87900400302056478FF792E
:10053D0000020564E9C313F9E813F8307C0EE96095
:10054D000278FFC3E81338F8E43400F9C3E894FFE8
:10055D00E99400400278FF885CD270206102A17C92
:10056D00741FF4552F4BF52FC274EB7002D27475B6
:10057D002A40307403752A0A306102A19020740359
:10058D0053DAFE207403752B20D0F0D0E0D0D0D2FA
:10059D00AD43E6103279010205C079030205C07939
:1005AD000A0205C0791E0205C079640205C079C82A
:1005BD000205C07817E4D5E0FDD8FAD9F6227A14F1
:1005CD007B780205E77A107B8C0205E77A0D7BB408
:1005DD000205E77A0B7BC80205E7E573D5E001223A
:1005ED007902E4C295D5E0FDD294D5E0FDC294D553
:1005FD00E0FDD295D5E0FDE920E002D29230E00297
:10060D00D296E573D5E0FDE920E002C29230E0021A
:10061D00C2967496D5E0FDD9C9EAF8D5E0FDD8FBB0
:10062D00DBB8C29522C37C007D0075F00005F0EAB1
:10063D0033FAEB33FB50F6EB13FBEA13FAC3E9FF86
:10064D00E8FEE89AF8E99BF95004EFF9EEF8B3ECFF
:10065D0033FCED33FDD5F0DFEDF9ECF822E889F050
:10066D008A20D2D4F8A9F07B0030F70B7BFFF4245D
:10067D0001F8E9F43400F9E88520F0A4ADF0F8E9CB
:10068D008520F0A4AFF0FEED2EF974003FFA7C0446
:10069D00C3EA13FAE913F9E813F8DCF48BF030F739
:1006AD000AE8F42401F8E9F43400F9E889F0C2D439
:1006BD00F8A9F0227882B60403020760C3E55C94C2
:1006CD0019401EE52D54067018206E367805799464
:1006DD00E7146007780A1460027812C3E541984068
:1006ED001F306E098564627569FF756A0185222464
:1006FD00E4F544F545F546F547F548C26E02076049
:10070D00D26E7994E7147013E523F43333F913F8AB
:10071D00E9540104F9E854FE020754E71414701467
:10072D00E523F4333333F913F8E9540304F9E854AA
:10073D00FC02075CE523F433333333F913F8E95442
:10074D00070404F9E854F8C39440F8E99400F988D3
:10075D0044894522C3E54113F9E54013F8C3E54447
:10076D0098F8E54599F9500CC3E89480E994FF4059
:10077D0016020798C3E8947FE99400500302079886
:10078D00787F7900020798788079FF8849894A2215
:10079D00E5492546F8E54A3547F9854A20E430070D
:1007AD0001F43548FA30E709C3EA94F04015020721
:1007BD00D6C3EA940F50030207D678FF79FF7A0F5C
:1007CD000207D6780079007AF0C3E5249561500AC6
:1007DD00C374019524500B0207F4E54A20E70E027D
:1007ED0007F4E54A30E706884689478A482278A506
:1007FD00E6FAC3E54933F8E54A33F912066AE930FA
:10080D00E70BC3E89480E994FF4013012FC3E894EC
:10081D007FE994005002012F787F7900012F7880B5
:10082D0079FFE820E715C3E52398F84009C3E8945C
:10083D000140030208567801020856E8F424012508
:10084D0023F8400302085678FF884B2278A6E6FA73
:10085D00A847A94812066AE930E70CC3E89401E9F4
:0E086D0094FF401602088BC3E894FFE9940044
:10087B00500302088B78FF790002088B780179FF0F
:10088B00E920E715C3E54B98F84009C3E89401400C
:10089B00030208B278010208B2E8F42401254BF8F0
:1008AB0040030208B278FF88242278FF2069287958
:1008BB00A1E76023E541601F74FF8541F084853912
:1008CB00F0306A0375F005A4F8C5F0600278FFC339
:1008DB00E895645002A864886322C3E54094C8E598
:1008EB00419400E56350031401F6046002F56322A2
:1008FB007883E6F520120F9375E8901205A275E840
:10090B009030EDFDA8BDA9BE12103A756E00756F43
:10091B0000C3740013FD7400606613FC74002CFCA0
:10092B0074003DFDECFAEDFBC3E89AE99B4014E53E
:10093B006E2400F56EE56F3400F56FEA2CFAEB3D93
:10094B00FB80E5AE6EAF6FC3E56F13F9E56E13F881
:10095B00C3E913F9E813F87A03C3E913F9E813F8B9
:10096B00DAF7AA201A7009756E00756F0002098BF1
:10097B001AEA6008EE28FEEF39FFDAF88E6E8F6FF9
:10098B002275E890227883E6FF30EDF9A8BDA9BE69
:10099B000570C3E57094084052757000E9FA79A0B0
:1009AB00E76044EA7007E571601B0209C4C3E89570
:1009BB00716010E5715006600C140209D00460F9E7
:1009CB000209D0E571F571C39472401B7561C0C308
:1009DB0094044013756180C39404400B756140C34C
:1009EB009404400375610075BB0822EFC39401604A
:1009FB001F7400601BC3E894FFE994035012C3E813
:100A0B00956EE9956F5009E561600C1561020A223C
:100A1B00E561F460020561A861C3E524985002A862
:100A2B0024C3E89562400AA862E562F4600385621C
:100A3B006188258826E570B4070375BB10227432D4
:100A4B0079A787F0A4C5F0A2F733F8C3E895614006
:100A5B0002A861882288248825882688642275400C
:100A6B00007541F022C2AF75C820A8CCA9CDAA3A17
:100A7B0030CF010A75C824D2AFC3EA13FAE913F9D0
:100A8B00E813F8AB3BAC3C883B893CC3E89BF8E9EB
:100A9B009C20690A547FF9306602618F41E9AD3DB4
:100AAB008A3DF9EA9D547FFA600678FF79FF41CEC3
:100ABB00AE3EAF3F8B3E8C3FA83BA93CC3E89EF8B4
:100ACB00E99FF9C3E54113FBE54013FAE82AF5402A
:100ADB00E93BF54150067540FF7541FF6136AA4071
:100AEB00AB41AC40AD417E047F02C3EB9404400D9F
:100AFB001E1FC3EB94084005206A021E1FC3ED1393
:100B0B00FDEC13FCDEF7C3EA9CFAEB9DFBEF6009EF
:100B1B00C3E913F9E813F8DFF7EA28FAEB39FB8A94
:100B2B00408B4150067BFF8B408B41C3EB940250B3
:100B3B0002D2663069047F0361617892E6FFC3E5F8
:100B4B0037948240110FC3E53794A040010FC3EFD8
:100B5B00940640027F057E02E541C4540FF9E5413E
:100B6B00C454F0F8E540C4540F28F8C3E89EFAE9E2
:100B7B009400FB4009C3EA9402EB940050047A0200
:100B8B00E4FB61DBAA40AB41EBC4FEEAC4540F4E5D
:100B9B00FCC3EA9CFAEB9400FBC3E813C313F8EA1B
:100BAB0028FAEB3400FB8A408B41C3EB94024002E2
:100BBB00C2667802EBC4FE7B00EAC4540F4EFAC344
:100BCB00EA98FA4005C3940250027A027892E6FF43
:100BDB0030600261DB855192855293D26043E6808F
:100BEB00C3E49AF8E49BF9C3E833F8E933F93066C8
:100BFB0002816EE8FAE9FBD3E913FDE813FC885197
:100C0B008952C3EF94036038EF20E00DE82CF8E92C
:100C1B003DF9ECFAEDFB020C37E828F8E939F9C39A
:100C2B00E82402F8E93400F97AFE7BFFC3EF940362
:100C3B00400E8A538B54884D894E8C4F8D5081A218
:100C4B00885389548A4D8B4E8C4F8D503069127559
:100C5B0053F07554FF754FF07550FF7551F0755289
:0F0C6B00FF81A2E8FAD3E813FC8851C3EF94038A
:100C7A006020EF20E007E82CF8ECFA818EE82824BF
:100C8A0002F87AFEC3EF940340088A53884D8C4FCA
:100C9A0081A288538A4D8C4FE568C3335002646B36
:100CAA00F56830600281AC753402D26043E680E5B3
:100CBA002D5406602DA840A941C3E913F9E813F899
:100CCA00306904E92440F9C2AF53E67F759100C345
:100CDA00E498F594E499F595759104D26043E68019
:100CEA00D2AF22D264754300752000306C037520A0
:100CFA0040020D0CD264754300752040306C0375B8
:100D0A00200078017901206620E52D54066002C290
:100D1A00647914E541C313700104F8C394144002C2
:100D2A007814306904781B791BC3E833F8C3E933B4
:100D3A00F9206010E543600C306903D53404D26DA4
:100D4A00A1C391B40543E59BF45440B52002A1AD7B
:100D5A0030690908C3E899400118A13B20640A08D0
:100D6A00C3E8994002A10CA13BC264C2AF53E67F1B
:100D7A007591003066127594007595F0759104D2DC
:100D8A006043E680D2AFA10CE5417EFFC333400940
:100D9A00C3334005C3334001FEC3E49E759400F596
:100DAA0095A186C3E53394015002A10C306402A1D7
:100DBA000CD802A1C1A13BC26DC2AF53E67F7591A7
:100DCA0000855394855495759104854D92854E936B
:100DDA00D26043E680D2AFE52D54066008206A024D
:100DEA000533020DFF306D0D206C0A206407158152
:100DFA0015810216CB2278003064027801E5377536
:100E0A00F007A4F9E5F028F5F0E9A2F013A2F1132E
:100E1A00A2F213F537C394785003753778C3E537D0
:100E2A0095384008D265C292C296C294306002C117
:100E3A0036854F92855093D26043E68022207D16F4
:100E4A00C2AF754202C295D293306202D296D2AF35
:100E5A00759F40021037C2AF754202C295D29730D1
:100E6A006202D292D2AF759F40021037307243208D
:100E7A007D20C2AF754203900165757B20C296C280
:100E8A0097306204D294C194D295D2AF759F410231
:100E9A001037C2AF754203900165757B20C292C2BA
:100EAA0093306204D294C1B4D295D2AF759F4302F3
:100EBA001037207D17C2AF754203900140C29630A9
:100ECA006202D294D2AF759F41021037C2AF754207
:100EDA0003900140C292306202D294D2AF759F430E
:100EEA00021037207D16C2AF754204C293D29730E2
:100EFA006202D294D2AF759F43021037C2AF7542D5
:100F0A0004C297D293306202D294D2AF759F410243
:100F1A001037307243207D20C2AF754205900154CC
:100F2A00757B08C294C295306204D292E13AD29398
:100F3A00D2AF759F40021037C2AF75420590017655
:100F4A00757B80C294C295306204D296E15AD297D8
:100F5A00D2AF759F40021037207D17C2AF75420588
:100F6A00900136C294306202D292D2AF759F40028B
:100F7A001037C2AF75420590014AC2943062EBD273
:100F8A0096D2AF759F40021037207D16C2AF7542C8
:100F9A0006C297D295306202D292D2AF759F4102B1
:100FAA001037C2AF754206C293D295306202D2960A
:100FBA00D2AF759F43021037307244207D20C2AFF2
:100FCA00754201900176757B80C292C293306204A9
:100FDA00D296E1E0D297D2AF759F43021037C2AFE3
:100FEA00754201900154757B08C296C2973062051A
:100FFA00D292021001D293D2AF759F4102103720CC
:10100A007D17C2AF75420190014AC292306202D284
:10101A0096D2AF759F43021037C2AF754201900155
:10102A0036C296306202D292D2AF759F41C2652211
:10103A00900134757B00C292C296C294C293C29741
:10104A00C295C26222788076070876070876010878
:10105A0076040876FF0876FF08760A08760208768C
:0F106A0001087601788C76010876000876B408C4
:1010790076FF0876FF0876FF0876030876FF08767C
:10108900010876FF0876250876D00876780876C8AC
:101099000876040876FF08760108760008767A084B
:1010A900760A0876010876010876000876FF087640
:1010B90000227887E6FFC272BF0302D2727888C223
:1010C9007DE630E102D27DC27E7889E630E102D246
:1010D9007EC3EF94026008758E01D2730210ED751C
:1010E9008E00C273227880E6149000809378A5F66A
:1010F9007881E6149000809378A6F67886E61490B5
:10110900008D9378A7F6789FE6F87005756B002136
:1011190034C3E8941140027811E82828F56B256B4F
:10112900256B28F56C256B2828F56D7886E6F53949
:10113900C394025003753902789CE67538FFB402EE
:10114900037538A0B4030375388278A3E6149000B8
:101159009A93F566113A22227896E6FA7897E6FB91
:101169007888E6B40305C3EB940EFB307F047A005C
:101179007BFFC3EB9AFCC3948250027C8275720098
:101189000572EC8572F0A4C3E5F0947D40F222D299
:101199007F31611205B11205B17A007B007C101212
:1011A90005A7E55C2AFA74003BFBDCF37C04C3EB7E
:1011B90013FBEA13FADCF7FEC27F316122757C006A
:1011C900757D00E5EF20E6037520000520903FFFBF
:1011D900E520146006901FFF1460009304600375F6
:1011E900EF1653D9BF7581C043FF801205A275EF71
:1011F9000643B203E5B3240220E70DF521E5E32018
:10120900E0068521B343E301113A7580FF75A40017
:1012190075F13075D4DF75900375A5FC75F2FC7511
:10122900D50175A60175E241C292C296C294120512
:10123900B6D293D297D2951205A2C293C297C295FC
:10124900113AE4F8F6D8FD756801114F121729789B
:10125900988673753001C2AF1205BB1205CB120512
:10126900B11205D21205B11205D91205B112185DD4
:101279001205BB1205BB1205B6C2AF757C00757DA0
:101289000078FA79FA308507D9FBD8F7021C0011E2
:10129900BB11EE3160316178988673113A75A900F6
:1012A90075B680757A0075881075890275C82475B8
:1012B900910475D84075A82275B80275E690759B9A
:1012C90080759D0075D10E75BCC075BB0875BA11C6
:1012D90075E8801205A2D2AF1208FB75360053DA01
:1012E900CF207E0343DA20307E0343DA1043DA014C
:1012F900C2D8C2711205BBD2617B037A0CE55B705F
:10130900077A0CDB030212821205B1207003021264
:1013190082C270E55CC3940240E1E52F541F855EEB
:101329005DF55EB55DD5DAD5C26153DACF207E03AE
:1013390043DA20307E0343DA10C2D8C27178A2E6BC
:101349007008D274E52F54E0F52FC2757529001283
:1013590005B6307409C3E529940A4002D27512050D
:10136900A778023074027800C3E55C9840F0C2AFF8
:101379001205CB1205CB1205CBD2AF1205BB754CAA
:10138900001205A7788CE6C394015003021477E58F
:1013990030C394015003021477757CA5757DF12043
:1013A9007435C3E55C94FF5003021477C2AF12058C
:1013B900E0D2AF1205B6C3E55C940150EFC2AF129B
:1013C90005CB1205AC1205CBD2AF1205B6C3E55C4D
:1013D90094FF40E90218E27F05D27F31611205B618
:1013E900C2AFC27F3161AE5CC3E55C947FD2AF50BE
:1013F9000281871205A2C2AF1205E0D2AFDFDA314E
:1014090098C3EE94057897F61205BB1218657F0A02
:10141900D27F31611205B6C2AFC27F3161AE5CC302
:10142900E55C947FD2AF50E61205A2C2AF1205CB9C
:101439001205AC1205CBD2AFDFD63198EE24037872
:1014490096F6F87997E7C394824003985006E82402
:10145900827897F61205BB1217761218941205B600
:0E1469003161C3E55C94FF500261A20218E2FB
:10147700757C00757D00C3E55C954C4003855C4C2D
:101487001205B678017988E7B403027805C3E55CED
:10149700984002618AC2AF1205E01205E01205E02A
:1014A700D2AF1205BB753000E4F531F5320531E5F1
:1014B70031F4703E0532789AE67819146012783262
:1014C70014600D787D14600878FA14600375320093
:1014D700C3E53298401C113A1205A2153275310046
:1014E70078998673C2AF1205E0D2AF7898867312E7
:1014F70005B61205ACE52A70053074024182780101
:101507002074027806C3E55C9840A21205B6E52A66
:101517007003021282C2AF113AE4F522F523F524D3
:10152700F525F526F567D2AF7885E6C333F565E48B
:10153700F544F545F546F547F548F570F52CF52DD5
:10154700F53775700875BB101205A212098C30EDBE
:10155700FDA8BDA9BEE97001F888711209907570E0
:101567000875BB1011BBC2AF7561FF120A4985220E
:1015770061852262852263D2AF75220175240175C8
:101587002501752601856069756A0175B69075A98B
:1015970003757A017888E6B40307C27D307602D2F4
:1015A7007DD268D269753300120F93120FC2120AE7
:1015B70069120A70120A69120A70120A69120CFE7D
:1015C7001206C1120E00120E47120A70120CED30ED
:1015D7006E031207612066031208B530660312080E
:1015E700E5120E00120E76120A70120CFE306E0310
:1015F70012079D120E00120EED120A70120CED303A
:101607006E031207FB120E00120F1C120A70120C47
:10161700FE306E03120859120E00120F93120A7051
:1016270012098C120CED120E00120FC21209901241
:101637000A7030692C856461856462856069756AA2
:101647000179187A0CC3E533994009C269D26A8ACD
:1016570035021668C3E55C940140030215C40216FF
:10166700D3306A25206C22E535147006C26AD26B26
:10167700A1C4F535C3E55C940140030215C478881D
:10168700E6C3940360030216D3753600C3E55F947F
:10169700014009856462856069756A0178FA79A4F1
:1016A700E760027803C3E55F985021307404E52AA8
:1016B700601A78F0306C058564617820C3E541983D
:1016C7005002A1C40536E55C6002C1D6753600C27A
:1016D700AF113A7887E6FE760211BB7887EEF6E41B
:1016E700F522F523F524F525F526F565752C007506
:1016F7002D0075A90075B680757A00D2AF1205B6B0
:10170700113A78A4E66006D293D295D29730740640
:10171700E52A70024182788DE6C394014002616731
:1017270081AF901A0D78201217B8E520B4A50CA345
:101737001217B8E520B45A03021756757CA5757DB4
:10174700F1114F121776757C00757D0002177590A1
:101757001A0378807B0A1217B8A308DBF9901A0FCF
:10176700788C7B191217B8A308DBF9901A2822C2C4
:10177700AF1217FB1217D8901A00740E1217BDA3D9
:1017870074091217BDA374151217BD901A03788038
:101797007B0A1217BCA308DBF9901A0F788C7B1908
:1017A7001217BCA308DBF912180F1217EC901A28AE
:1017B70022E493F622E6438F01538FFDFFC3E583AF
:1017C700941C400122EF857CB7857DB7F0538FFECF
:1017D70022438F02438F01857CB7857DB7901A0D11
:1017E700F0538FFC22901A0D74A5F1BD901A0E7458
:1017F7005AF1BD227A3079D07820901A401217B862
:10180700E520F709A3DAF6227A3079D0901A40E773
:101817001217BD09A3DAF822AB74A875BB010279C8
:1018270080BB02027981BB03027982BB04027994EF
:10183700BB05027983BB06027986BB07027992BB97
:1018470008027987BB0902799CBB0A027988BB0B1E
:10185700027989E8F7227C051205BBDCFB22C2AFBF
:0F1867001205CB1205D21205D91205E01205ACFD
:101876001205CB1205D21205D91205E01205AC12DB
:1018860005CB1205D21205D91205E0D2AF22C2AF9E
:101896001205E01205D91205D21205CB1205AC12BB
:1018A60005E01205D91205D21205CB1205AC1205B8
:1018B600E01205D91205D21205CBD2AF22AE74AF13
:1018C60075C2AF1205CB1205CB1205CB1205ACDEE5
:1018D600F21205E01205ACDFF8D2AF221165115DF8
:1018E600115D75740175750175760011C37C05ADC2
:1018F6005C1205BBC3ED955C70F5C3E55C940140D5
:101906000AC3E55C94FF403302191F111F121776B4
:101916001165C2AF75EF16115DDCD40576C3E576A9
:101926009403500280C5115D0575E5741490009FFF
:1019360093F808C3E57598500280AD115D115D05F9
:1019460074C3E574940C5002809B12104F121776E4
:07195600C2AF75EF16115D31
:0319FD000211C60E
:101A00000E091507070104FFFF0A020101A55A018B
:101A100000B4FFFFFF03FF01FF25D078C804FF01DA
:091A200000FF0A010100FF00FFB4
:101A400023475F556C74726132304123202020207F
:101A500023424C48454C492346333930232020202B
:101A60002020202020202020202020202020202076
:101C0000C2AFC2D353D9BF7581C043B20343FF8073
:101C1000752438752503B1DC7529A5752AF175E29F
:101C20004043F12053A4DF75D4FFD2857DFA7803B9
:101C300079E67C10752200752300901DE97B0675FE
:101C400024987525013085028145208508D8FBD967
:101C5000F9DCF781B7308508D8FBD9F9DCF781B713
:101C6000B19CE493A3C39A6004DDC381B7DBDBB10D
:101C70008E6002812E7B08E493FAA3B16FDBF87AC1
:101C800030B16F752200752300B18EEAFCEBFDC305
:101C9000ED94FE400EB18E8A278B28ED30E0048A49
:101CA000828B83B18E7AC270D8C3ED94FE601950D6
:101CB000CEBD002BEC600F7520007521FF7529004B
:101CC000752A000200008100A827A9280809D80465
:101CD000D90281DCB192EA89AAF281CE0D81A3C337
:101CE000ED94035053EDA2E092007AC5C3E58294CF
:101CF00000E583941C508A200010438F02438F011B
:101D00008529B7852AB7F0300029A827A92808090E
:101D1000438F01538FFDD804D902A133C3E58394C7
:101D20001C4003A3A11689AAE28529B7852AB7F02A
:101D3000A3A116538FFC817F7AC1BD030CE493A34A
:101D4000FAB153DCF8B14B817F8181AA22AB23B178
:101D50006FEBFAEA6222752608C3E52313F523E543
:101D60002213F52250066323A0632201D526EAB18F
:101D7000DCB1DC75260AEAF4200102D285300102CA
:101D8000C285B1DCC3134002C201D526EB22B19259
:101D9000EAFB208502A192308502A197752608AE44
:101DA00024AF25C3EF13FFEE13FEB1E0B1DCC3EAAD
:101DB000133085024480FA30E703632201C3E52330
:101DC00013F523E52213F52250066323A0632201B5
:101DD000D526D9E52265236523F52222AE24AF2539
:101DE0000E0FDEFEDFFCD20122424C48656C6934E6
:071DF000373164F390060196
:00000001FF
